:020000040000FA
:060000004DEF20F012009C
:0600080004EF10F01200ED
:060018000CEF10F01200D5
:062000004DEF20F012007C
:022006001200C6
:062008003EEF19F012008A
:0620180045EF19F0120073
:02201E000100BF
:0C202000B640000060000000410000001D
:04202C00D9CFE6FF23
:10203000E1CFD9FFE652A394676A656A6A6A010E26
:10204000E66EE66AE66A6B0EE66E0F0EE66E13EC5F
:1020500020F00B6E050EE15E0B50160E626E9F0EA9
:10206000666E7B0E646EDF6ADF500B6E0C6A080EC4
:102070000B5C000E0C5810E2DF50040DF3CFE9FFAB
:10208000F4CFEAFF000EE926040EEA22EE6AEE6AB9
:10209000EE6AEE6ADF2AE8D7608C636A6098609C1B
:1020A00065A607D065960001B46BB96BBA6BBB6BC4
:1020B000F7D70001010ECB6FCC6FCD6BCE6BC16B30
:1020C000DF6A020EDF5C26E2EA6ADF34FE0BEA36E4
:1020D000E96EAC0EE926000EEA22EE6AED6AEA6AC3
:1020E000DF34FE0BEA36E96EA80EE926000EEA227E
:1020F000EE6AED6ADF50EA6AC50FE96E000EEA2269
:10210000EF6ADF50EA6AC70FE96E000EEA22EF6A53
:10211000DF2AD7D70001080EAC6F040EAD6F160E84
:102120006A6E0401200E026F040E036F080E016F29
:10213000840E006F0001A26BA16BE552E552E7CF60
:10214000D9FF1200D9CFE6FFE1CFD9FFE652000157
:10215000A1510FE1606A646A160E626E9F0E666E90
:102160007B0E646E60B602D06086FCD70001010E63
:10217000A16FA10508E160BA06D0656A646A64804F
:102180006488020EA16F6550040B06E06450040BD6
:1021900003E065947DEC16F060B258D06550010BF9
:1021A00008E06450010B05E041DF0001040EA16F5F
:1021B00065906550100B06E06450100B03E068EC6E
:1021C00016F0659865AC19D064AC0FD0010EE66EC0
:1021D000E66A000EE66EE66A730EE66EE66A8CEC60
:1021E0001EF00B6E060EE15E0B50659C0001C9519E
:1021F00001E0C907C95101E1DFD96550200B05E0B5
:102200006450200B02E04FEC16F06550020B13E017
:102210006450020B10E0010EE66EE66A000EE66EF8
:10222000E66AE6687F0EE66E8CEC1EF00B6E060E1C
:10223000E15E0B50676A040E0001E76EA119E8AE7B
:1022400002D0E73402D0E750A15D02E2A49439D075
:1022500064A636D0DF6A040EDF5C32E265A630D0B9
:1022600061CFC2F00001C251780BE842E842E84277
:10227000C36F6596C2B506D0C351EA6AC70FE96E4F
:10228000000E05D0C351EA6AC50FE96E000EEA22BE
:10229000EF70C35103E194EC16F010D0000EE66E1F
:1022A000E66AC20EE66E000EE66E720EE66EE66A34
:1022B0008CEC1EF00B6E060EE15E0B50DF2ACBD7C6
:1022C000A494E552E552E7CFD9FF1200D9CFE6FF3B
:1022D000E1CFD9FF020EE126FD0EDBA407D0E66AAE
:1022E000FE0EDBCFE6FFF7D9E552E552FD0EDBA28D
:1022F00008D0010EE66EFE0EDBCFE6FFECD9E5520C
:10230000E552FE0EDB500C6A6A0F0B6E0F0E0C22AC
:102310000BC0DEFF0CC0DDFFDECFE9FFDDCFEAFF43
:10232000FD0EDBCFEFFF020EE15C02E2E16AE55257
:10233000E16EE552E7CFD9FF1200D9CFE6FFE1CF3A
:10234000D9FF020EE126FD0EDB500AE0FE0EEA6A1E
:10235000DB34FE0BEA36E96EAC0EE926000E09D03E
:10236000FE0EEA6ADB34FE0BEA36E96EA80EE926B9
:10237000000EEA22EECFDEFFEDCFDDFFD9CFE9FF81
:10238000DACFEAFFEE50ED1003E1F36AF46A44D0CD
:10239000DECFE9FFDDCFEAFF020EE926000EEA22DA
:1023A000FB0EDBCFEEFFFC0EDBCFEDFFDECFE9FF58
:1023B000DDCFEAFFEE52FA0EDBCFEFFF400EDECFAD
:1023C000E9FFDDCFEAFFE850EF16880EDECFE9FF28
:1023D000DDCFEAFFE850EF12FD0EDB500AE0FE0E03
:1023E000EA6ADB34FE0BEA36E96EAC0EE926000E33
:1023F00009D0FE0EEA6ADB34FE0BEA36E96EA80E5F
:10240000E926000EEA22EF74DECF0BF0DDCF0CF0F0
:102410000BC0F3FF0CC0F4FF020EE15C02E2E16AC4
:10242000E552E16EE552E7CFD9FF1200D9CFE6FFC2
:10243000E1CFD9FF020EE126FE0EDB5020E1A6C05F
:10244000E9FFA7C0EAFFEE52080EEF6EA6C0E9FF53
:10245000A7C0EAFF020EE926000EEA22200EEE6E69
:10246000040EED6EA6C0E9FFA7C0EAFF8C0EEF6E6A
:10247000ACC0E9FFADC0EAFF840EEF6E3BD0FD0EAD
:10248000DB50E8240D6EFE0EDB50040DF3500D24DE
:10249000040DF3CF0BF0F4CF0CF0000E0B26040E5E
:1024A0000C220BC0DEFF0CC0DDFF840EDECFE9FF87
:1024B000DDCFEAFFE850EF12FD0EDB50E8240D6E91
:1024C000FE0EDB50040DF3500D24010F040DF3CF6D
:1024D0000BF0F4CF0CF0000E0B26040E0C220BC0F8
:1024E000DEFF0CC0DDFF840EDECFE9FFDDCFEAFFAB
:1024F000E850EF12020EE15C02E2E16AE552E16EA1
:10250000E552E7CFD9FF1200D9CFE6FFE1CFD9FFDF
:1025100060A84ED0FE0EEA6ADB34FE0BEA36E96EA6
:10252000AC0EE926000EEA22EE50EFCFEAFFE96E8C
:10253000400EEE16EE6AEE6AEE6AFE0EEA6ADB34D2
:10254000FE0BEA36E96EAC0EE926000EEA22EE50EA
:10255000EFCFEAFFE96EEE7CFE0EEA6ADB34FE0B9B
:10256000EA36E96EAC0EE926000EEA22EF74400E60
:102570000B6EFE0EEA6ADB34FE0BEA36E96EAC0E39
:10258000E926000EEA22EE50EFCFEAFFE96E0B508B
:10259000EF16FE0EEA6ADB34FE0BEA36E96EAC0E8D
:1025A000E926000EEA22EE50EFCFEAFFE96EEF7C5B
:1025B000E552E7CFD9FF12000001CB514DE1010EEA
:1025C000CB6FCC5149E1010ECC6F020EB15D0DE134
:1025D000ACC0E9FFADC0EAFFEE52EF6AACC0E9FF64
:1025E000ADC0EAFFC80EEF6E1200B10535E1C46B55
:1025F000A4C0E9FFA5C0EAFFEE52080EEF6EA4C02A
:10260000E9FFA5C0EAFF020EE926000EEA22200E2D
:10261000EE6E040EED6EA4C0E9FFA5C0EAFF840EC5
:10262000EF6E010EC46FA6C0E9FFA7C0EAFFEE522D
:10263000080EEF6EA6C0E9FFA7C0EAFF020EE9266A
:10264000000EEA22200EEE6E040EED6EA6C0E9FF2B
:10265000A7C0EAFF800EEF6E12000001CD6BCE6BBB
:10266000020EB15D18E1A6C0E9FFA7C0EAFFEE5275
:10267000080EEF6EA6C0E9FFA7C0EAFF020EE9262A
:10268000000EEA22280EEE6E040EED6EA6C0E9FFE3
:10269000A7C0EAFF1DD0B5510401265D0001B65167
:1026A0000401275904E226C4B5F027C4B6F0CAD8FD
:1026B000ACC0E9FFADC0EAFF020EE926000EEA2237
:1026C000280EEE6E040EED6EACC0E9FFADC0EAFF61
:1026D000C80EEF6E1200D9CFE6FFE1CFD9FF020E90
:1026E000E126000EDE6E040EDD6EFD0EDB50E824EA
:1026F0000D6EFE0EDB50040DF3500D24040DF4CFCF
:102700000CF0D9CFE9FFDACFEAFFF350EE260C50F8
:10271000ED22DECFE9FFDDCFEAFFEF9EFD0EDB50BD
:102720000AE1FE0EEA6ADB34FE0BEA36E96EA80E19
:10273000E926000E09D0FE0EEA6ADB34FE0BEA360B
:10274000E96EAC0EE926000EEA22DECFEEFFDDCF09
:10275000EDFFDECFE9FFDDCFEAFFEF9CDECFE9FF43
:10276000DDCFEAFF040EE926000EEA22EF8C020E0E
:10277000E15C02E2E16AE552E16EE552E7CFD9FFA2
:10278000120060980001B4BF2BD0B9AF09D0020E7F
:10279000B16FCE5101E161DF0001CC6BCB6B120058
:1027A000A6C0E9FFA7C0EAFFEE52080EEF6EA6C072
:1027B000E9FFA7C0EAFF020EE926000EEA22200E7A
:1027C000EE6E040EED6EA6C0E9FFA7C0EAFF8C0E08
:1027D000EF6EACC0E9FFADC0EAFF840EEF6E1200F1
:1027E000040120AF0DD00001010EB16FCD5101E108
:1027F00034DF0001CC6BCB6BCA5123E1DCEF12F06C
:102800000001020EB16FA6C0E9FFA7C0EAFFEE52B9
:10281000080EEF6EA6C0E9FFA7C0EAFF020EE92688
:10282000000EEA22200EEE6E040EED6EA6C0E9FF49
:10283000A7C0EAFF840EEF6ECC6BCB6BCA5101E1EF
:10284000BBDE1200D9CFE6FFE1CFD9FFE652080E7A
:10285000DF6E0001B55D000EB6590AE2B5C0DFFFBC
:10286000B05102E1010E03D0B00502E1020EB06FDB
:10287000DF500C6AE850B55DB56F0C50B659B66FB5
:10288000ACC0E9FFADC0EAFFEE52DFCFEFFF280E8C
:10289000BE6F040EBF6FB4B118D0DF502DE0B2C0D0
:1028A000F6FFB3C0F7FFB22B000EB3230800F550BC
:1028B000E66EBEC0E9FFBFC0EAFFBE2B000EBF231D
:1028C000E552E750EF6EDF06E8D7DF5015E0B2C003
:1028D000E9FFB3C0EAFFB22B000EB323EF50E66E60
:1028E000BEC0E9FFBFC0EAFFBE2B000EBF23E5520A
:1028F000E750EF6EDF06E9D7E552E552E7CFD9FFA3
:102900001200D9CFE6FFE1CFD9FF020EE126A4C025
:10291000E9FFA5C0EAFFEE52EFCFDFFFDFCF0BF0FC
:102920000B500001BA5D000EBB5902E2BAC0DFFFD6
:10293000DF500B6E0C6AE850BA5DBA6F0C50BB5991
:10294000BB6F010EDB6ADF50F36E010EDBCFF4FFCD
:10295000F350F45C16E2010EDB50EA6A280FE96ED0
:10296000040EEA22EF50E66EB7C0E9FFB8C0EAFFF6
:10297000B72B000EB823E552E750EF6E010EDB2AAD
:10298000E2D7000ED880BA55000EBB5527E2A6C08C
:10299000E9FFA7C0EAFFEE52080EEF6EA6C0E9FFFE
:1029A000A7C0EAFF020EE926000EEA22280EEE6E0C
:1029B000040EED6EA4C0E9FFA5C0EAFFEF50400B86
:1029C00006E1A6C0E9FFA7C0EAFFC80E05D0A6C071
:1029D000E9FFA7C0EAFF880EEF6E28D0A6C0E9FF86
:1029E000A7C0EAFFEE52080EEF6EA6C0E9FFA7C02F
:1029F000EAFF020EE926000EEA22200EEE6E040E19
:102A0000ED6EA6C0E9FFA7C0EAFF840EEF6EBC51D1
:102A1000BD1107E005D0BDC0FAFF0001BC51F96E41
:102A2000FADF0001B99FCA5101E1C6DD020EE15C87
:102A300002E2E16AE552E16EE552E7CFD9FF12000A
:102A4000D9CFE6FFE1CFD9FFE6520001B48F010EE6
:102A5000E66EE66AE66A6B0EE66E0F0EE66E13EC45
:102A600020F00B6E050EE15E0B50200EE66EE66A5E
:102A7000E66A000EE66E040EE66E13EC20F00B6EB6
:102A8000050EE15E0B50608CDF6A020EDF5C10E227
:102A9000DF50EA6AC50FE96E000EEA22EF6ADF50E6
:102AA000EA6AC70FE96E000EEA22EF6ADF2AEDD765
:102AB000010EE66EE66AE66AA30EE66E000EE66EAC
:102AC00013EC20F00B6E050EE15E0B50609C0001D4
:102AD000080EAC6F040EAD6F000EA46F040EA56F50
:102AE000A4C0A6F0A76F22C4A2F0A25102E1100E6A
:102AF00012D0010EE66EE66AA20EE66E000EE66EDB
:102B0000010EE66EE66A8CEC1EF00B6E060EE15EC0
:102B10000B500001200EA16FE552E552E7CFD9FF1F
:102B20001200800E0401205D58E10001C00EB46F58
:102B300004012351030A2FE0010A09E0030A4BE1D3
:102B40000001EC0EB26F3D0EB36F120E3ED022515B
:102B5000F66EF76AD890F636F736BA0EF6263E0EBF
:102B6000F7220900F5CFB2F00A00F5CFB3F0020E5C
:102B70000001F76AB225F66EB351F7220800F5CFCF
:102B8000B5F0030EF76AB225F66EB351F7220800CE
:102B9000F5CFB6F01200030E225D1AE22251F66E56
:102BA000F76AD890F636F736BC0EF6263E0EF722B8
:102BB0000900F5CFB2F00A00F5CFB3F0B2C0F6FFCE
:102BC000B3C0F7FF0800F5500001B56FB66B1200F7
:102BD0000001B46B12000001B46B1200D9CFE6FF04
:102BE000E1CFD9FF020EE1260401286B296B2051A9
:102BF0001F0B020A11E0030A0CE0010A3CE100018C
:102C0000B48F040128810001C00535E10401288347
:102C100032D00001B48F2FD00001B48F040124BF43
:102C20000BD024510F0BE96EEA6AD890E936EA36E8
:102C3000A80EE926000E0AD024510F0BE96EEA6AAD
:102C4000D890E936EA36AC0EE926000EEA22EECF3D
:102C5000DEFFEDCFDDFFDECFE9FFDDCFEAFFEF5096
:102C6000800B09E0DECFE9FFDDCFEAFFEF50040B78
:102C700002E0010E286F0001B4AF07D0280EB26F3A
:102C8000040EB36FB481020EB56F020EE15C02E276
:102C9000E16AE552E16EE552E7CFD9FF12006AA082
:102CA00015D0A4C0E9FFA5C0EAFFEF5080080DE1F0
:102CB000ACC0E9FFADC0EAFFEF50840806E1A4C054
:102CC000E9FFA5C0EAFF8C0EEF6E6A90659A1200CC
:102CD0006484659860820001010EC16F000EE66E8B
:102CE000E66AE66EE66A750EE66EE66A8CEC1EF043
:102CF0000B6E060EE15E0B5012000001C16B000E60
:102D0000E66EE66AE66EE66A740EE66EE66A8CECDD
:102D10001EF00B6E060EE15E0B506092649465A48B
:102D200002D06594FCD71200D9CFE6FFE1CFD9FFDE
:102D3000E65200012D0EC96FFD0EC21553E17E0E45
:102D4000C215E8407F0B040DF3CFA4F0F4CFA5F03B
:102D5000000EA427040EA523A4C0A6F0A5C0A7F0CA
:102D6000A675A4C0E9FFA5C0EAFFEF503C0BE842FE
:102D7000E8420D0835E1DF6A080EDF5C23E2A4C0FB
:102D8000E9FFA5C0EAFF020EE926000EEA22EE5096
:102D9000EFCFEAFFE96EEF50E66EDF50EA6A200FF0
:102DA000E96E040EEA22E552E750EF6EA4C0E9FF97
:102DB000A5C0EAFF020EE926000EEA22EE2AEF2263
:102DC000DF2ADAD7A4C0E9FFA5C0EAFF020EE92690
:102DD000000EEA22200EEE6E040EED6E0DD807D026
:102DE0003AD805D0FD0EC215040801E159D8E552C4
:102DF000E552E7CFD9FF12000001B06BCA6BCD6B73
:102E0000CE6BC46BB16BACC0E9FFADC0EAFFEF9E07
:102E1000AC75ACC0E9FFADC0EAFFEF9EAC75A6C0D3
:102E2000E9FFA7C0EAFFEF9EB46BB56BB66BB96B59
:102E3000BA6BBB6B8CD8000EE66EE66AE66EE66A8D
:102E4000030EE66EE66A8CEC1EF00B6E060EE15E7B
:102E50000B50C1EF13F0020E0001B15D02E181EFF2
:102E600014F0B16BC4511AE1A6C0E9FFA7C0EAFF94
:102E7000EE52080EEF6EA6C0E9FFA7C0EAFF020EF1
:102E8000E926000EEA22200EEE6E040EED6EA6C0BC
:102E9000E9FFA7C0EAFF8C0EEF6E1200C46B1200B0
:102EA000D9CFE6FFE1CFD9FFE652ACC0E9FFADC014
:102EB000EAFFEF50400B01E0010EDF6E0001AC7540
:102EC000080EA15D08E122C463FF635002E0100E0A
:102ED00001D0040EA16FB10526E1ACC0E9FFADC081
:102EE000EAFF020EE926000EEA22280EEE6E040E1C
:102EF000ED6EA8DC020E0001B05D06E1ACC0E9FF9A
:102F0000ADC0EAFF840E0DD0DF5006E1ACC0E9FF92
:102F1000ADC0EAFFC80E05D0ACC0E9FFADC0EAFF06
:102F2000880EEF6E0FD0B9AF0CD0BC51BD1107E0C9
:102F300005D0BDC0FAFF0001BC51F96EFADF0001F7
:102F4000B99FB16BE552E552E7CFD9FF12000401FA
:102F50002051600BE842E842E842E842E8420009BA
:102F600001E0120021510C0A50E00B0A3FE00C0A6C
:102F700031E0010A22E00B0A1EE0020A1CE0030A0B
:102F800018E0080A10E0010A0CE00F0A08E0030A42
:102F900001E012000001B48F080EA16F120091EF42
:102FA00015F020EF15F00001A20EB26F000EB36F06
:102FB0000CD0EEEF15F006EF18F024510001B26FBF
:102FC000B36BA30EB227000EB323B481010EB56F0D
:102FD000B48F12000001B48F04012451EA6AA30FD8
:102FE000E96E000EEA2222C4EFFF1200000EE66E28
:102FF000E66AE66EE66A020EE66EE66A8CEC1EF0A3
:103000000B6E060EE15E0B5012001200D9CFE6FFE8
:10301000E1CFD9FF050EE1260401220510E1205180
:103020001F0B00090CE10001B48F030E0401215DA8
:1030300004E10001010EC06F02D00001C06B040169
:10304000225101E011D120511F0B020801E00CD1E7
:1030500024510F0B000901E107D124510F0B010886
:1030600001E202D1200E0001A15D01E0FDD0B48F8C
:10307000040124BF16D024510F0BE96EEA6AD890E0
:10308000E936EA36A80EE926000EEA22EECFDEFF88
:10309000EDCFDDFF24510F0BEA6AC70FE96E000E7A
:1030A00015D024510F0BE96EEA6AD890E936EA365A
:1030B000AC0EE926000EEA22EECFDEFFEDCFDDFFFB
:1030C00024510F0BEA6AC50FE96E000EEA22020EC8
:1030D000EFCFDBFFD950020FE96EDACFEAFFEF50F6
:1030E000010B03E1000EDF9401D0DF8424BF0BD07D
:1030F00024510F0BE96EEA6AD890E936EA36A80E39
:10310000E926000E0AD024510F0BE96EEA6AD89026
:10311000E936EA36AC0EE926000EEA22DECFEEFFF3
:10312000DDCFEDFF030E215D20E1DECFE9FFDDCF36
:10313000EAFFEF50800B11E024BF07D024510F0BA2
:10314000EA6AC70FE96E000E06D024510F0BEA6A37
:10315000C50FE96E000EEA22EF82840EDECFE9FF92
:10316000DDCFEAFFE850EF127FD0DF74DECFE9FF5A
:10317000DDCFEAFFEF50800B1BE0DECFE9FFDDCFB4
:10318000EAFFEF9EDECFE9FFDDCFEAFFEF8C020E14
:10319000E66EE66ADECFE6FFDDCFE6FF050EE66E01
:1031A000E66A8CEC1EF00B6E060EE15E0B5005D04D
:1031B000DECFE9FFDDCFEAFFEF8CDF74D950020FDD
:1031C000E96EDACFEAFFEF50020B07E1DECFE9FF4D
:1031D000DDCFEAFFEF50800B2BE0040124BF07D0C6
:1031E00024510F0BEA6AC70FE96E000E06D0245176
:1031F0000F0BEA6AC50FE96E000EEA22EF923B0E52
:103200000B6EDECFE9FFDDCFEAFFE850EF16020ECE
:10321000E66EE66ADECFE6FFDDCFE6FF050EE66E80
:10322000E66A8CEC1EF00B6E060EE15E0B5007D0CA
:103230003B0EDECFE9FFDDCFEAFFE850EF160401D9
:1032400024510F0B0C6A6A0F0B6E0F0E0C22030E2B
:103250000BC0DBFF040E0CC0DBFF030EDBCFE9FF6E
:10326000040EDBCFEAFFEF90050EE15C02E2E16ABB
:0C327000E552E16EE552E7CFD9FF1200F5
:04327C00DACFE4FFC2
:10328000E652E552E5CFDAFF1100D8CFE4FFE0CFF8
:10329000E4FFE46EDACFE4FFE652E552E5CFDAFF71
:1032A000E550E5CFE0FFE5CFD8FF100004D8A2EC51
:1032B00010F032D8FCD70F0EC112800E9B6E700E2C
:1032C000D36E100ED26ED2AEFED7B50EE96E0F0ED3
:1032D000EA6E900EEF6E02D816EF10F0F19E856840
:1032E0000F015B6B5C6B5D6B5E6B5F6B92689368F1
:1032F000F80E946E95689668806A816A826A836A1D
:10330000846A896A8A6A8B6A8C6A8D6A0001E16BB9
:10331000E26BE36BE46B1200200E0001E76EA11973
:10332000E8AE02D0E73402D0E750A15D05E360507B
:10333000020B01E0120048D81200D9CFE6FFE1CF1E
:10334000D9FFFE0EDB50A96EA69EA69CA680A850B3
:10335000E552E7CFD9FF1200D9CFE6FFE1CFD9FF81
:10336000FE0EDB50A00805E1F40EF36EFE0EF3CF67
:10337000DBFFFE0EDBCFE6FFE0DFE552E552E7CFF5
:10338000D9FF1200D9CFE6FFE1CFD9FFE652A00E58
:10339000DF6EE00EDF5C11E2DFCFE6FFCEDFE5524D
:1033A0000B6EFE0EDB500B5C05E1DF28E66EC5DF21
:1033B000E55205D0020EDF24EBD7FE0EDB50E552BE
:1033C000E552E7CFD9FF1200D9CFE6FFE1CFD9FF11
:1033D000090EE126FE0EF36E060EF3CFDBFF070E9D
:1033E000DB68080EDB68DF6ADFCF0BF0140EE76ED8
:1033F0000B18E8AE02D0E73402D0E7500B5C01E3D3
:1034000099D0060EDB50926E070EDB50956E080EBB
:10341000DB50400DF3503809946E080EDB40E84055
:103420003F0BFC09966E080EDB50020D080EF3CF21
:10343000DBFFDB80070EDBBE05D0FE0EF36E080E51
:10344000F3CFDBFF070EDB50020D070EF3CFDBFFE0
:10345000DB80060EDBBE05D0FE0EF36E070EF3CF4B
:10346000DBFF060EDB50020D060EF3CFDBFFDB8029
:10347000010EE66E2DEC20F0E552811CE76E020E87
:10348000E7CFDBFFDFCFE9FFEA6AE9BEEA68600E5B
:10349000E926000EEA22EF50E66EDFCFE9FFEA6A86
:1034A000E9BEEA68750EE926000EEA22E552E75009
:1034B000EF6EDFCFE9FFEA6AE9BEEA68600EE9264F
:1034C000000EEA22EF6A010EDB6ADBCF0BF0080E7A
:1034D000E76E0B18E8AE02D0E73402D0E7500B5C81
:1034E00027E2020EDBCFE6FF010EF36EDB5004E0B5
:1034F000D890F336E806FCE1F350E552E71415E006
:10350000010EF36EDB5004E0D890F336E806FCE1E0
:10351000F3500B6EDFCFE9FFEA6AE9BEEA68600E9E
:10352000E926000EEA220B50EF12010EDB2ACDD75E
:10353000DF2A5AD70001746B84B402D0010E746F75
:10354000F80EE66EFADEE552000901E1A1D0DF6A6D
:10355000DFCF0BF0140EE76E0B18E8AE02D0E734A5
:1035600002D0E7500B5C20E2E00EDF24E66EE5DEE1
:10357000E5520B6EDFCFE9FFEA6AE9BEEA68600E4A
:10358000E926000EEA22EF500B14E66EDFCFE9FFCA
:10359000EA6AE9BEEA688A0EE926000EEA22E552E6
:1035A000E750EF6EDF2AD4D7DF6ADFCF0BF0140EBF
:1035B000E76E0B18E8AE02D0E73402D0E7500B5CA0
:1035C00067E2020EDB6A010EDB6ADBCF0BF0140E42
:1035D000E76E0B18E8AE02D0E73402D0E7500B5C80
:1035E0003AE2010EDB50DF5C33E0010EDBCFE9FF96
:1035F000EA6AE9BEEA688A0EE926000EEA22EFCFFF
:103600000BF0DFCFE9FFEA6AE9BEEA688A0EE92635
:10361000000EEA22EF500B1410E0010A0EE0030A3C
:103620000CE0060A0AE00C0A08E0180A06E0300A74
:1036300004E0600A02E0C00A04E1010EF36E020E2B
:1036400002D0020EF36EF3CFDBFFDB50020803E083
:10365000010EDB2ABAD7020EDB50020817E1DFCFDA
:10366000E9FFEA6AE9BEEA68750EE926000EEA2279
:10367000EF50E66EDFCFE9FFEA6AE9BEEA68600E66
:10368000E926000EEA22E552E750EF6EDF2A8DD7D9
:10369000DF6ADFCF0BF0080EE76E0B18E8AE02D042
:1036A000E73402D0E7500B5C0CE2DFCFE9FFEA6AB7
:1036B000E9BEEA68000EE926050EEA22EF6ADF2A73
:1036C000E8D7020EF36E040EF3CFDBFF050EDB6AC4
:1036D000DF6ADFCF0BF0150EE76E0B18E8AE02D0F5
:1036E000E73402D0E7500B5C01E394D0010EDB6AB3
:1036F000DBCF0BF0080EE76E0B18E8AE02D0E73414
:1037000002D0E7500B5C01E383D0010EDBCFE6FF74
:10371000080EDF02F350E552E724E76E020EE7CF12
:10372000DBFF010EF36EDB5004E0D890F336E806C1
:10373000FCE1F3500B6EDFCFE9FFEA6AE9BEEA680D
:10374000600EE926000EEA22EF500B145EE0F50E43
:10375000E66EF3DDE552F36E020EDB50F35C06E13C
:10376000010EF36E050EF3CFDBFF4FD0020EDBCF61
:10377000E6FFF2DDE552E76E030EE7CFDBFF000167
:10378000F35109E0030EDBCFE6FFFCDDE552E76E07
:10379000030EE7CFDBFF030EDB50FF0836E0E00E41
:1037A000F36E030EDBCFF4FFF350F45C12E3030E71
:1037B000DB50E7080EE3030EDB50200F0B6E010E0B
:1037C0000B5204E0E846FE0B0B06FCE1050100137A
:1037D0001CD0040EDBCF0BF0080EE76E0B18E8AE22
:1037E00002D0E73402D0E7500B5C0FE2040EDBCFCF
:1037F000E9FFEA6AE9BEEA68000EE926050EEA2258
:10380000030EDBCFEFFF040EDB2A010EDB2A70D79D
:10381000DF2A5FD7050EDBCFF3F0F90EE66E8DDD04
:10382000E552000901E1F1D0DF6ADFCF0BF0080EAD
:10383000E76E0B18E8AE02D0E73402D0E7500B5C1D
:103840000CE2DFCFE9FFEA6AE9BEEA68000EE9268A
:10385000050EEA22EF6ADF2AE8D7DF6ADFCF0BF036
:10386000150EE76E0B18E8AE02D0E73402D0E75031
:103870000B5C01E3CAD0010EDB6ADBCF0BF0080E54
:10388000E76E0B18E8AE02D0E73402D0E7500B5CCD
:1038900001E3B9D0010EDBCFE6FF080EDF02F350E3
:1038A000E552E724E76E020EE7CFDBFF010EF36E71
:1038B000DB5004E0D890F336E806FCE1F3500B6EE1
:1038C000DFCFE9FFEA6AE9BEEA68600EE926000E8A
:1038D000EA22EF500B1401E193D0020EDB50F00B03
:1038E000E8380F0BE76E030EE7CFDBFFDB5005E197
:1038F000270EF36E040EF3CFDBFF030EDBCF0BF0CE
:10390000000EE76E0B18E8AE02D00B3403D0E75080
:10391000D8800B5414E2030EDBCF0CF00A0EE76ED6
:103920000C18E8AE02D0E73402D0E7500C5C07E296
:10393000030EDB501D0FE76E040EE7CFDBFF030E17
:10394000DBCF0BF00A0EE76E0B18E8AE02D0E734BF
:1039500002D0E7500B5C07E3030EDB50FA0FE76E73
:10396000040EE7CFDBFF040EDBCF02F5020EDB50C7
:103970000F0BE76E030EE7CFDBFFDB5005E1270EF1
:10398000F36E040EF3CFDBFF030EDBCF0BF0000E64
:10399000E76E0B18E8AE02D00B3403D0E750D880A6
:1039A0000B5414E2030EDBCF0CF00A0EE76E0C187A
:1039B000E8AE02D0E73402D0E7500C5C07E2030E19
:1039C000DB501D0FE76E040EE7CFDBFF030EDBCFEE
:1039D0000BF00A0EE76E0B18E8AE02D0E73402D007
:1039E000E7500B5C07E3030EDB50FA0FE76E040EA3
:1039F000E7CFDBFF040EDBCF03F505012C0E046FD0
:103A0000010EDB2A3AD7DF2A29D70001E151E21162
:103A100002E1000E08D0E1C0E9FFE2C0EAFFEF508A
:103A2000800B01E0010E000967E1010EDB6ADF6A2D
:103A3000DFCF0BF0080EE76E0B18E8AE02D0E734CC
:103A400002D0E7500B5C1CE2DFCFE9FFEA6AE9BE77
:103A5000EA68EB0EE926000EEA22EFCF0BF0DFCF8B
:103A6000E9FFEA6AE9BEEA68000EE926050EEA22E5
:103A7000EF500B5C03E0DE52010EDD6EDF2AD8D77B
:103A8000010EDB0413E1080EE66E000EE66E050E75
:103A9000E66E010EE66EE66E9DEC11F00B6E050E05
:103AA000E15E0B50F3CFE1F0F4CFE2F0DF6ADFCF5D
:103AB0000BF0080EE76E0B18E8AE02D0E73402D028
:103AC000E7500B5C19E2DFCFE9FFEA6AE9BEEA687A
:103AD000000EE926050EEA22EF50E66EDFCFE9FF81
:103AE000EA6AE9BEEA68EB0EE926000EEA22E55230
:103AF000E750EF6EDF2ADBD70001E351E41102E16A
:103B0000000E08D0E3C0E9FFE4C0EAFFEF50800BED
:103B100001E0010E00094CE1F70EE66E9DEC19F094
:103B2000E55200090FE1F60EE66E9DEC19F0E55244
:103B3000000904E10501081D070B26D0070E050149
:103B4000081522D0F60EE66E9DEC19F0E55200093C
:103B50000DE10501081D040BE8407F0B0C6E081DEC
:103B6000020BE8240B6E081D010B0CD0040E05019E
:103B70000815E8407F0B0C6E020E0815E8240B6E4A
:103B8000010E08150B100C108B6E010EE66E080E60
:103B9000E66E050EE66EE66A010EE66E9DEC11F02D
:103BA0000B6E050EE15E0B50F3CFE3F0F4CFE4F0C3
:103BB000090EE15C02E2E16AE552E16EE552E7CF0F
:103BC000D9FF12008150100B01E0010E0001CF5D02
:103BD00007E08150100B01E0010ECF6F81A8010CAE
:103BE000000C8150200B01E0010E0001D05D07E0C8
:103BF0008150200B01E0010ED06F81AA010C000C56
:103C000000019F51A01104E1100E9F6F270EA06FBD
:103C10009F07000EA05B60A207D09F51A0112EE16C
:103C20008C708CB013D027D00001A15102E18C9090
:103C300022D0A10502E18C8009D0020EA15D02E133
:103C40008C8019D0040EA15D03E18C908C8212004F
:103C5000100EA15D06E100019F51A0110FE18C70D3
:103C60000AD0200EA15D0AE100019F51A01106E1DA
:103C70008C708CA002D08C9212008C8212008C90DE
:103C80008C92130ED36E1200700ED36ED2AEFED78E
:103C900012001200120061EF1FF012001E0EE66EFD
:103CA000010EE66E66EC11F0E552E552010EE66E8D
:103CB000080EE66E050EE66EE66A010EE66E9DECF7
:103CC00011F00B6E050EE15E0B50F3CFE3F0F4CF75
:103CD000E4F012000001C0051EE10001C1051BE176
:103CE000D3DF60920001C16B0001100EF46F0E0E65
:103CF000F56FF407000EF55BF451F511FAE16084FD
:103D0000080EF46F070EF56FF407000EF55BF45123
:103D1000F511FAE160941200D9CFE6FFE1CFD9FFA7
:103D2000FD0EDBCF06F0FE0EDBCF07F0050E06180A
:103D300001E1075036E0E868061802E17F0E071837
:103D40002FE0030E061801E1075028E0020E0618C6
:103D500001E1075021E0010E061801E107501AE0C9
:103D6000740E061801E1075013E0750E061801E104
:103D700007500CE0730E061801E1075005E0720EC3
:103D800006180FE107500DD084DF0BD078DF09D083
:103D90007BDF07D083DF05D080DF03D07CDF01D05D
:103DA00079DF010EE552E7CFD9FF12000001280E9E
:103DB000B76F040EB86F080EBA6FBB6BC80EBC6F3E
:103DC0003D0EBD6FB98F1200040128A103D08C8075
:103DD0008C8202D08C908C920001E66BE00EE76F33
:0C3DE000220EE86F020EE96FEA6B120081
:043DEC0012010002BE
:103DF00000000008D804550001000102000109027A
:103E00002900010100E03209040000020301010061
:103E1000092111010001223F00070581030800016B
:103E2000070501030800010403090434034D006978
:103E300000630072006F006300680069007000207A
:103E40000054006500630068006E006F006C006F36
:103E50000067007900200049006E0063002E001CFE
:103E6000034B006500790062006F0061007200641E
:103E7000002000440065006D006F0005010906A1E7
:103E800001050719E029E71500250175019508814D
:103E90000295017508810395057501050819012929
:103EA0000591029501750391039506750815002586
:103EB000E70507190029E78100C0FE3D273E2B3E9C
:023EC0005F3E63
:0E3EC200040120511F0B010801E012002451E1
:103ED00001E01200060E215D1BE12351230A18E0C8
:103EE000010A0CE0030A14E10001A20511E100013E
:103EF000100EB26F3E0EB36F090E06D000017B0E9E
:103F0000B26F3E0EB36F3F0EB56FB66BC00EB46F9F
:103F100004012051600BE842E842E842E842E842EE
:103F2000010801E0120021510B0A28E0080A1BE0F9
:103F3000090A13E0080A07E00B0A03E0080A23E075
:103F40001200D6EF1EF00001300EB26F040EB36FF8
:103F5000010EB56FB66BC10E0FD00001800EB46FAD
:103F600023C430F412000001310EB26F040EB36F9F
:103F7000010EB56FB66B810EB46F12000001800E9A
:083F8000B46F22C431F41200F9
:083F88001E0EF66E200EF76E0E
:103F9000000EF86E00010900F550FB6F0900F550A6
:103FA000FC6F03E1FB6701D03DD00900F550F66FCF
:103FB0000900F550F76F0900F550F86F0900090086
:103FC000F550E96E0900F550EA6E09000900090094
:103FD000F550F96F0900F550FA6F09000900F6CFA6
:103FE000FDF0F7CFFEF0F8CFFFF0F6C0F6FFF7C018
:103FF000F7FFF8C0F8FF0001F95302E1FA5307E0B8
:104000000900F550EE6EF907F8E2FA07F9D7FDC09E
:10401000F6FFFEC0F7FFFFC0F8FF0001FB07000E30
:06402000FC5BBFD712009B
:0A402600FE0EE3CFE9FFFF0EE3CF2B
:10403000EAFFE9CFF3FFEACFF4FFFB0EE35003E121
:10404000FC0EE35009E0FB0EE30602E2FC0EE30681
:0A405000FD0EE350EE6EF1D71200F2
:06405A00FF0EE3500E6EA4
:10406000480E01D04C0EE76EE72EFED7E76AE72E2A
:0A407000FED70E2EF7D70000120055
:06407A00000EF36E00EEE3
:1040800000F0080E01D81200EA6002D0EE6AFCD7F8
:0A409000F350E9601200EE6AFCD75D
:06409A0013EE00F023EE1E
:1040A00000F0F86A0A9CC4EC1FF003EC10F056EC28
:0640B00019F0FBD712001D
:0A40B6000000000000000000000000
:1040C00000000000000000000000000000000000F0
:1040D00000000000000000000000000000000000E0
:1040E00000000000000000000000000000000000D0
:0740F00000000000000000C9
:020000040030CA
:0100000021DE
:0100010008F6
:010002001FDE
:010003003EBE
:010005009169
:01000600A158
:0200000400F00A
:10000000FFFFFF352A4C4939292B504F51524628C2
:10001000FF3E89FF100D1824273D2E2D110B1C23A8
:100020002C3C3032050A1722873B2F341909152141
:10003000383A1333060708203726120F1B161A1FEB
:1000400036250C0E1D04141EFFFFFFFFE2E1E0FF4A
:10005000FFFFFFFFFFFFFFFFFFFFFFFFFFFFFFFFB0
:10006000FFFFFFFFFFFFFFFFFFFFFFFFFFFFFFFFA0
:10007000FFFFFFFFFFFFFFFFFFFFFFFFFFFFFFFF90
:10008000FFFFFFFFFFFFFFFFFFFFFFFFFFFFFFFF80
:10009000FFFFFFFFFFFFFFFFFFFFFFFFFFFFFFFF70
:1000A0002F52344F335038510F49374E0E4A364D88
:1000B0000C46124713482A4C2B3930491E3A1F3B35
:1000C000203C213D223E233F244025412642274318
:1000D0002D442E45FFFFFFFFFFFFFFFFFFFFFFFF48
:1000E000F8FFF6FFFFFFFFFFFF70000000000000B9
:1000F00000000000FF0700000000FFFFFFFFFFFF00
:00000001FF
